:10000000E2010108000801080008010800080108D1
:10001000000801080008010800080108000801089C
:10002000000801080008010800080108000801088C
:10003000000801080008010800080108000801087C
:10004000000801080008010800080108000801086C
:10005000000801080008010800080108000801085C
:10006000000801080008010800080108000801084C
:10007000000801080008010800080108000801083C
:10008000000801080008010800080108000801082C
:10009000000801080008010800080108000801081C
:1000A000000801080008010800080108000801080C
:1000B00000080108000801080008010800080308FA
:1000C00001080108000801080008010800080108EB
:1000D00000080108000801080008010800080108DC
:1000E00000080108000801080008010800080108CC
:1000F00000080108000801080008010800080108BC
:1001000000080108000801080008010800080108AB
:10011000000801080008010800080108000801089B
:10012000000801080008010800080108000801088B
:10013000000801080008010800080108000801087B
:10014000000801080008010800080108000801086B
:10015000000801080008010800080108000801085B
:10016000000801080008010800080108000801084B
:10017000000801080008010800080108000801083B
:1001800001080400040C2800FF0C2900020C0500E3
:10019000000C060066002506CB0A2507CD0AA90239
:1001A000090200092600DE096600BF0C890043072A
:1001B000DB0AFF0C29002506DB0ACD0A08022A000B
:0A01C00000000000EA02E00A000857
:0207FE00C10A2E
:00000001FF
